:030000000219FDE5
:03000B000200AA46
:03002B0002018A45
:03005B0002034756
:0300730002033451
:1000800002030406080C10182030406080040608A3
:100090000C10182030406080A0C00003070F1F0D17
:1000A0000D04050D050305030302C2AF306308C24A
:1000B0006385798AD2AF32C0D0C0E0206221E525C5
:1000C0006016E473E525F4C3334009758A00D263F2
:1000D000F57901D6F58AD262D0E0D0D0D2AF32C362
:1000E000E526334009758A00D263F57901F0F58A77
:1000F000C262E526F4603030682620720DD0E0D070
:10010000D0C295C294C293D2AF32C295C294C29368
:10011000206F0D20660A7414D5E0FDE57BF4529043
:10012000D0E0D0D0D2AF32758A00D263757900C2E8
:100130008DD262212001C4306805206602D295016B
:10014000C4306805206602D29401C4306805206678
:1001500002D29301C4D29230680A2066077410D587
:10016000E0FDD29501C4D29130680A206607741070
:10017000D5E0FDD29401C4D290D29230680A2066B4
:10018000077410D5E0FDD29301C4C2AFC2AD53E6EF
:10019000EFC0D0C0E0D2D3D2AFE57A6009E5776096
:1001A0000575770041E1757701C2CEE52A60072029
:1001B0007449152A21FB7800790020742EE58030DF
:1001C0007E01F430E70278FF53DACF207E0343DA72
:1001D00020307E0343DA10C2D8C271E580307E0140
:1001E000F430E70279FFC3E89970CB306103752AD8
:1001F00018207403752A18885CD27020740DE52BC2
:100200006004152B410B43DA01C2D8207002417AF9
:10021000A85C206102C2702074367982B70431C3B1
:10022000E894F0400374F0F8E8C4540F28F8798497
:10023000B703024150C313C3138721200802C3131D
:10024000200A06C3C898F8415028F8500374FFF8F4
:100250008822E52D54066022206B1FE536C333C388
:1002600033F8E564C313C313F9C39522400289220E
:10027000E82522F52250037522FF7882B6045985BD
:100280002224A824C3E52495614002A861C3E8950F
:10029000634002A8638825E566700241CBC3E8AAE3
:1002A000669A5003E8FAE4F9EAC333FBE568F45BC5
:1002B00029400D2567F8E56760021567400B41CBC3
:1002C0000AC3E5679A5002056778FF8826C26FC3A4
:1002D000E52694F84002D26FC3E52594404002D24F
:1002E0006420CF0AD0E0D0D043E610D2AD32C2CFE6
:1002F000053AE57A6009E5786005757800612A7548
:1003000078017801E52A6005307402152AC3E55C9E
:1003100094014005755F00612A756000756900E50C
:100320005F2401F55F5003755FFFD0E0D0D043E656
:1003300010D2AD32C2AF53E67F7592FA7593FFC209
:1003400060759104D2AF32C2AF53E6EFC2ADC0D0F8
:10035000C0E0C0F0D2D3D2AFA8FBA9FCE57A600719
:10036000C3E913F9E813F8C2D830710261B953DA5E
:10037000CF207E0343DA10307E0343DA20D271E5CA
:1003800080307E01F420E702619088278928A1E669
:1003900053DACF207E0343DA20307E0343DA10C2E3
:1003A000D8C271307402A1D27800E580307E01F4A9
:1003B00030E702A1D2885CA1BA53DACF207E034392
:1003C000DA20307E0343DA10C27120610281925339
:1003D000DACF207E0343DA10307E0343DA20C2D81E
:1003E000D27188578958C3E89555F8E99556F97B35
:1003F000007E087A00C3E8948CE994005005755B90
:10040000008184882178A2E6A8216055C3E894C8B9
:10041000E994005008E4D2E4FB7A0A815FC3E894CF
:1004200068E994015008E4D2E3FB7A0F815FC3E8E6
:1004300094D0E994025008E4D2E2FB7A1E815FC3B3
:10044000E894A0E994055008E4D2E1FB7A3C815F8E
:10045000C3E89498E994085008E4D2E0FB7A787EE7
:1004600000C3E89559FCE9955AFD30E70AECF424FD
:0F04700001FCEDF43400FD755B00C3EC9AED9ECA
:10047F005003755B018859895A85575585585678A9
:10048F0002A1BAC3E89527F8E99528F9307C02A1B3
:10049F009E307B02A19E307A02A19720750281B512
:1004AF00E9FDE8FC81D4E9C313F9E813F8307902C8
:1004BF00A197E9C313F9E813F8307802A197E9C3BC
:1004CF0013FDE813FC20612CC3EC941CED94024047
:1004DF000281EBED701EC3EC94C850180529E52975
:1004EF0070021529C3E529940A5002A1D2755C0048
:1004FF00D270A1D2E529600215297888E6F9740037
:10050F00207F087896B90302789EE624FAFEE43439
:10051F0000FFC3EC9EFCED9FFD9208B90310A208EB
:10052F005007207609D276A13D307602C276A20816
:10053F005016B9030DECF42401FCEDF43400FD0268
:10054F00055778007900A19EB90315EC33FCED3304
:10055F00FDC3EC940AFCED9400FD50047C007D007B
:10056F00C3EC94FFED9400400678FF7900A19EEC58
:10057F008572F0A4C5F0A2F733F8790040030205A5
:10058F00BA78FF79000205BAE9C313F9E813F83016
:10059F007C0EE9600278FFC3E81338F8E43400F901
:1005AF00C3E894FFE99400400278FF885CD2702082
:1005BF006102A1D2741FF4552F4BF52FC274EB704B
:1005CF0002D274752A18307403752A0A306102A199
:1005DF00E620740353DAFE207403752B06D0F0D097
:1005EF00E0D0D0D2AD43E61032790102061679037E
:1005FF00020616790A020616791E02061679640299
:10060F00061679C80206167817E4D5E0FDD8FAD990
:10061F00F6227A147B7802063D7A107B8C02063D17
:10062F007A0D7BB402063D7A0B7BC802063D790238
:10063F00E4D291D5E0FDD294D5E0FDC294D5E0FD92
:10064F00C291D5E0FDE920E002D29530E002D293CD
:10065F00E573D5E0FDE920E002C29530E002C293D8
:10066F007496D5E0FDD9C9EAF8D5E0FDD8FBDBBE1D
:10067F00D29122C37C007D0075F00005F0EA33FAB9
:10068F00EB33FB50F6EB13FBEA13FAC3E9FFE8FE7B
:10069F00E89AF8E99BF95004EFF9EEF8B3EC33FC64
:1006AF00ED33FDD5F0DFEDF9ECF822E889F08A2083
:1006BF00D2D4F8A9F07B0030F70B7BFFF42401F8BC
:1006CF00E9F43400F9E88520F0A4ADF0F8E98520CD
:1006DF00F0A4AFF0FEED2EF974003FFA7C04C3EAEC
:1006EF0013FAE913F9E813F8DCF48BF030F70AE8A2
:1006FF00F42401F8E9F43400F9E889F0C2D4F8A938
:10070F00F0227882B6040302076CC3E55C940140C3
:10071F0003020736852224E4F544F545F546F547EF
:10072F00F548C26E02076C7882E6FCD26EE522F5C0
:10073F0023783879C7AA40AB41C3EB13FBEA13FA0E
:10074F00EC146013C3EB13FBEA13FAEC14146007F9
:10075F00C3EB13FBEA13FAD1828844894522C3E520
:10076F00449523F8E5459400F9500CC3E89480E9CB
:10077F0094FF401602079DC3E8947FE9940050034D
:10078F0002079D787F790002079D788079FF88495D
:10079F00894A22E5492546F8E54A3547F9854A2031
:1007AF00E4300701F43548FA30E709C3EA94F04022
:1007BF00150207DBC3EA940F50030207DB78FF79BA
:1007CF00FF7A0F0207DB780079007AF0C3E52495F2
:1007DF0061500AC374019524500B0207F9E54A20B2
:1007EF00E70E0207F9E54A30E706884689478A4847
:1007FF002278A5E6FAC3E54933F8E54A33F912063C
:10080F00BAE930E70BC3E89480E994FF4013013451
:10081F00C3E8947FE9940050020134787F79000196
:10082F0034788079FFE820E715C3E52398F840096D
:10083F00C3E89401400302085B780102085BE8F407
:10084F0024012523F8400302085B78FF884B2278A8
:10085F00A6E6FAA847A9481206BAE930E70CC3E89A
:0F086F009401E994FF4016020890C3E894FFE952
:10087E009400500302089078FF79000208907801E6
:10088E0079FFE920E715C3E54B98F84009C3E894D2
:10089E000140030208B778010208B7E8F4240125E5
:1008AE004BF840030208B778FF88242278FFC26411
:1008BE0020693D206A12D264C3E541940A4009C3FF
:1008CE00E52594405002C26479A1E76023E54160BA
:1008DE001F74FF8541F0848539F0306A0375F00589
:1008EE00A4F8C5F0600278FFC3E895645002A864CE
:1008FE00886322C3E54094C8E5419400E563500344
:10090E00142112046002F5632202091A2275E8907E
:10091E00227883E6FFE5E820ECF7A8BDA9BE0570B6
:10092E00C3E57094084052757000E9FA79A0E7604B
:10093E0044EA7007E571601B020955C3E8957160C2
:10094E0010E5715006600C140209610460F9020989
:10095E0061E571F571C39472401B7561C0C3940457
:10096E004013756180C39404400B756140C39404B9
:10097E00400375610075BB0622E5612410500274B8
:10098E00FFF5617982B7040221AEC3A861E5249810
:10099E005002A824C3E895634002A86388258826E0
:1009AE00E570B4070375BB1022743279A787F0A4E3
:1009BE00C5F0A2F733F8C3E895614002A86188221A
:1009CE008824882588268864227540007541F02287
:1009DE00C2AF75C820A8CCA9CDAA3A30CF010A75EE
:1009EE00C824D2AFC3EA13FAE913F9E813F8AB3B04
:1009FE00AC3C883B893CC3E89BF8E99C20690A54CF
:100A0E007FF930670241F84155AD3D8A3DF9EA9DC7
:100A1E00547FFA600478FF79FFAE3EAF3F8B3E8C79
:100A2E003FA83BA93CC3E89EF8E99FF9C3E54113F3
:100A3E00FBE54013FAE82AF540E93BF5415006750F
:100A4E0040FF7541FF419FAA40AB41AC40AD417E96
:100A5E00047F02C3EB940440021E1FC3EB940840B4
:100A6E00021E1FC3ED13FDEC13FCDEF7C3EA9CFA66
:100A7E00EB9DFBEF6009C3E913F9E813F8DFF7EA22
:100A8E0028FAEB39FB8A408B4150067BFF8B408B5B
:100A9E0041C3EB94025002D2673069047F0341CA0E
:100AAE007892E6FFC3E537948240110FC3E5379481
:100ABE00A040010FC3EF940640027F057E02E54180
:100ACE00C4540FF9E541C454F0F8E540C4540F285E
:100ADE00F8C3E89EFAE99400FB4009C3EA9402EBDE
:100AEE00940050047A02E4FB6144AA40AB41EBC48B
:100AFE00FEEAC4540F4EFCC3EA9CFAEB9400FBC30F
:100B0E00E813C313F8EA28FAEB3400FB8A408B4152
:100B1E00C3EB94024002C2677802EBC4FE7B00EA8C
:100B2E00C4540F4EFAC3EA98FA4005C39402500219
:100B3E007A027892E6FF30600261448551928552C6
:100B4E0093D26043E680C3E49AF8E49BF9C3E8339A
:100B5E00F8E933F930670261D7E8FAE9FBD3E91314
:100B6E00FDE813FC88518952C3EF94036038EF20DF
:100B7E00E00DE82CF8E93DF9ECFAEDFB020BA0E8EC
:100B8E0028F8E939F9C3E82402F8E93400F97AFEC5
:100B9E007BFFC3EF9403400E8A538B54884D894ECE
:100BAE008C4F8D50810B885389548A4D8B4E8C4FB0
:100BBE008D503069127553F07554FF754FF07550A6
:100BCE00FF7551F07552FF810BE8FAD3E813FC88DC
:100BDE0051C3EF94036020EF20E007E82CF8ECFA05
:100BEE0061F7E8282402F87AFEC3EF940340088ADE
:100BFE0053884D8C4F810B88538A4D8C4FE568C3BB
:100C0E00335002646BF5683060028115753402D280
:100C1E006043E680E52D5406602DA840A941C3E946
:100C2E0013F9E813F8306904E92440F9C2AF53E62A
:100C3E007F759100C3E498F594E499F59575910448
:100C4E00D26043E680D2AF22D26575430075200094
:100C5E00306C03752040020C75D26575430075200B
:0E0C6E0040306C03752000780179012067206A
:100C7C00E52D54066002C2657914E541C313700179
:100C8C0004F8C3941440027814306904781B791B5F
:100C9C00C3E833F8C3E933F9206010E543600C3046
:100CAC006903D53404D26DA12C911D0543E59B54E9
:100CBC0040B52002A11630690908C3E89940011813
:100CCC0081A420650A08C3E8994002817581A4C2F9
:100CDC0065C2AF53E67F759100306712759400754D
:100CEC0095FC759104D26043E680D2AF8175AE401D
:100CFC00AF41C3EE33FEEF33FF50047EFF7FFFC3E3
:100D0C00E49EF594E49FF59581EEC3E53394015090
:100D1C000281753065028175D802A12A81A4C26D49
:100D2C00C2AF53E67F7591008553948554957591A8
:100D3C0004854D92854E93D26043E680D2AFE52D6B
:100D4C0054066008206A020533020D68306D0D20D0
:100D5C006C0A206507158115810216072278003070
:100D6C0064053065027801E53775F007A4F9E5F004
:100D7C0028F5F0E9A2F013A2F113A2F213F537C390
:100D8C0094785003753778C3E53795384008D266A8
:100D9C00C295C294C293306002A1A2854F92855035
:100DAC0093D26043E68022207D16C2AF754202D2F8
:100DBC0091C292306202D293D2AF759F11020FAAE8
:100DCC00C2AF754202D291C290306202D295D2AFBC
:100DDC00759F11020FAA307245207D22C2AF754259
:100DEC0003900166757B02C293D290D2923062045A
:100DFC00D294C102C291D2AF759F01020FAAC2AFA9
:100E0C00754203900166757B02C295D292306204E2
:100E1C00D294C122C291D2AF759F21020FAA207D1C
:100E2C0017C2AF754203900141C293306202D29453
:100E3C00D2AF759F01020FAAC2AF75420390014158
:100E4C00C295306202D294D2AF759F21020FAA20B4
:100E5C007D16C2AF754204D292C290306202D29417
:100E6C00D2AF759F21020FAAC2AF754204D290D2A5
:100E7C0092C292306202D294D2AF759F01020FAA35
:100E8C00307243207D20C2AF754205900155757BB1
:100E9C0004C294D291306204D295C1AAC292D2AF4C
:100EAC00759F11020FAAC2AF754205900177757B31
:100EBC0001C294D291306204D293C1CAC290D2AF13
:100ECC00759F11020FAA207D17C2AF7542059001C4
:100EDC0037C294306202D295D2AF759F11020FAA1D
:100EEC00C2AF75420590014BC2943062EBD293D2E3
:100EFC00AF759F11020FAA207D18C2AF754206D2A2
:100F0C0090D292C291306202D295D2AF759F0102FB
:100F1C000FAAC2AF754206D292C291306202D2932E
:100F2C00D2AF759F21020FAA307245207D20C2AF2F
:100F3C00754201900177757B01C295D292306204A3
:100F4C00D293E152C290D2AF759F21020FAAC2AFC9
:100F5C00754201900155757B04C293D290D29230A8
:100F6C006204D295E174C292D2AF759F01020FAAAE
:100F7C00207D17C2AF75420190014BC295306202C1
:100F8C00D293D2AF759F21020FAAC2AF75420190C6
:100F9C000137C293306202D295D2AF759F01C266FF
:100FAC0022900135757B00C295C294C293D292D225
:100FBC0091D290C26222788076090876090876046C
:100FCC000876FF0876030876FF08760A0876030889
:100FDC007601087601788C76010876FF0876FF0892
:100FEC0076FF0876FF0876FF0876030876FF08760A
:100FFC00FF0876FF0876250876D008762808765004
:10100C000876040876FF08760208760008767A08D7
:10101C0076FF0876010876010876000876030876D4
:10102C0000227887E6FFC272BF0302D2727888E68C
:10103C00C394036008C27DE630E102D27DC27E78A3
:10104C0089E630E102D27EC3EF94026008758E010E
:10105C00D273021066758E00C273227880E61490EB
:0E106C0000809378A5F67881E61490008093BA
:10107A0078A6F67886E61490008D9378A7F6788697
:10108A00E6F539C394025003753902789CE675383F
:10109A00FFB402037538A0B4030375388278A3E657
:1010AA001490009A93F566120FAD22227896E6FA0A
:1010BA007897E6FB7888E6B40305C3EB940EFB3019
:1010CA007F047A007BFFC3EB9AFCC3948250027CB4
:1010DA00827572000572EC8572F0A4C3E5F0947D06
:1010EA0040F222D27F11B61206077A007B007C10EA
:1010FA001205FDE55C2AFA74003BFBDCF37C04C3B1
:10110A00EB13FBEA13FADCF7FEC27F11B622E5EF16
:10111A0020E6037520000520903FFFE520146006B5
:10112A00901FFF1460009304600375EF1253D9BF38
:10113A007581C043FF801205F875EF0243B203E5DB
:10114A00B3240220E70DF521E5E320E0068521B36B
:10115A0043E301120FAD7580FF75A40075F1907518
:10116A00D47F75908775A5BF75F2BF75D50075A632
:10117A000175E241120FADE4F8F6D8FD7568011267
:10118A000FC212166078988673753001C2AF1206C4
:10119A001112062112060712062812060712062F36
:1011AA00120607C2AF78FA79FA308707D9FBD8F75F
:1011BA00021C00112E116711B511B67898867312A8
:1011CA000FAD75A90075B680757A00758810758996
:1011DA000275C82475910475D84075A82275B8029D
:1011EA0075E690759B80759D0075D10E75BC587516
:1011FA00BB0675BA1175E8801205F8D2AF12091745
:10120A0075360053DACF207E0343DA20307E03435B
:10121A00DA1043DA01C2D8C271120611D2617B0315
:10122A007A0CE55B70077A0CDB030211AD12060734
:10123A002070030211ADC270E55CC3940240E1E57F
:10124A002F541F855E5DF55EB55DD5DAD5C2615353
:10125A00DACF207E0343DA20307E0343DA10C2D885
:10126A00C27178A2E67008D274E52F54E0F52FC255
:10127A007575290012060C307409C3E529940A40D1
:10128A0002D2751205FD78023074027800C3E55C5B
:10129A009840F0C2AF120621120621120621D2AFDF
:1012AA00120611754C007888E6B40302618C1205A7
:1012BA00FD788CE6C39401500302138CE530C39485
:1012CA0001500302138C207435C3E55C94FF50036C
:1012DA0002138CC2AF120636D2AF12060CC3E55CFB
:1012EA00940150EFC2AF120621120602120621D251
:1012FA00AF12060CC3E55C94FF40E90218087F02AE
:10130A00D27F11B612060CC2AFC27F11B6AE5CC351
:10131A00E55C947FD2AF40741205F8C2AF1206366C
:10132A00D2AFDFDC11EDC3EE7897F6120611121672
:10133A00A212178B7F0AD27F11B612060CC2AFC255
:10134A007F11B6AE5CC3E55C947FD2AF50E612055E
:10135A00F8C2AF120621120602120621D2AFDFD658
:10136A0011EDEE24037896F61206111216A2121740
:10137A00BA12060C11B6C3E55C94FF500241D002C2
:10138A001808C3E55C954C4003855C4C12060C7842
:10139A00017988E7B403027805C3E55C9840024105
:1013AA00B0C2AF120636120636120636D2AF12068F
:1013BA0011753000E4F531F5320531E531F4703F4D
:1013CA000532789AE67819146012783214600D782A
:1013DA007D14600878FA146003753200C3E5329808
:1013EA00401D120FAD1205F8153275310078998635
:1013FA0073C2AF120636D2AF7898867312060C12F1
:10140A000602E52A700530740221AD7801207402C3
:10141A007806C3E55C9840A17888E6C39403600324
:10142A0012060CE52A70030211ADC2AF120FADE429
:10143A00F522F523F524F525F526F567D2AF78854B
:10144A00E6C333F565E4F544F545F546F547F54851
:10145A00F570F52CF52DF53775700875BB1012056A
:0E146A00F812091BE5E820ECFBA8BDA9BEE9BD
:101478007001F8887112091F75700875BB10112E5C
:10148800C2AF7561FF1209B7852261852262852284
:1014980063D2AF7522017524017525017526018572
:1014A8006069756A0175B69075A903757A017888BF
:1014B800E6B40307C27D307602D27DD268D2697560
:1014C8003300120F03120F341209D71209DE120962
:1014D800D71209DE1209D7120C67120711120D690B
:1014E800120DB31209DE120C56306E0312076D206E
:1014F80067031208BA306703120901120D69120D49
:10150800E21209DE120C67306E031207A2120D698F
:10151800120E5B1209DE120C56306E03120800120E
:101528000D69120E8C1209DE120C67306E03120858
:101538005E120D69120F031209DE12091B120C56F6
:10154800120D69120F3412091F1209DE3069328533
:101558006461856462856069756A0179187A0CC36B
:10156800E53399400FC269D26A8A3585646185641A
:1015780063021589C3E55C940140030214DF021677
:101588000F306A1D206C1AE535147006C26AD26BDA
:1015980081DFF535C3E55C940140030214DF0216D0
:1015A8000F75360078FA79A4E760027803C3E55F1F
:1015B800985054307404E52A604D7888E6B40317CF
:1015C800207D05207607A1DF307602A1DF206C0799
:1015D800D26C856461A11E78F0306C0585646178F1
:1015E80020C3E54198500281DF306C1BC26CC27D7C
:1015F800307602D27DD26A75351285646181DF0545
:1016080036E55C6002C112753600C2AF120FAD78C4
:1016180087E6FE7602112E7887EEF6E4F522F523AA
:10162800F524F525F526F565752C00752D0075A9A9
:101638000075B680757A00D2AF12060C120FAD781D
:10164800A4E66006C292C291C290307409C3E5361E
:101658009404400221AD61BE901A0D78201216E460
:10166800E520B4550CA31216E4E520B4AA0302162B
:1016780082120FC21216A20216A1901A0378807B5A
:101688000A1216E4A308DBF9901A0F788C7B19125A
:1016980016E4A308DBF9901A2822C2AF1217231206
:1016A80016FD901A00740E1216E9A374061216E9B4
:1016B800A374151216E9901A0378807B0A1216E8AB
:1016C800A308DBF9901A0F788C7B191216E8A30887
:1016D800DBF9121736121714901A2822E493F6220F
:1016E800E6438F01538FFD75EF0275B7A575B7F106
:1016F800F0538FFE22438F02438F0175EF0275B7B7
:10170800A575B7F1901A0DF0538FFC22901A0D743D
:1017180055D1E9901A0E74AAD1E9227A3079D07895
:1017280020901A40D1E4E520F709A3DAF7227A30AD
:1017380079D0901A40E7D1E909A3DAF922AB74A865
:1017480075BB01027980BB02027981BB03027982F1
:10175800BB04027984BB05027986BB06027992BB79
:1017680007027987BB080279A3BB0902799CBB0AE7
:10177800027988BB0B027989E8F7227C05120611E9
:10178800DCFB22C2AF12062112062812062F12060F
:101798003612060212062112062812062F120636E3
:1017A80012060212062112062812062F120636D237
:1017B800AF22C2AF12063612062F120628120621D1
:1017C80012060212063612062F12062812062112D7
:1017D800060212063612062F120628120621D2AF6A
:1017E80022AE74AF75C2AF1206211206211206216D
:1017F800120602DEF2120636120602DFF8D2AF2215
:1018080012178B121783121783757401757501757A
:1018180076001217E97C05AD5C120611C3ED955CE4
:1018280070F5C3E55C9401400AC3E55C94FF40375A
:1018380002184C1217451216A212178BC2AF75EF79
:1018480012121783DCD10576C3E576940350028023
:10185800C11217830575E5741490009F93F808C3A7
:0F186800E57598500280A8121783121783057434
:10187700C3E574940C50028094120FC21216A2C2D0
:07188700AF75EF1212178389
:0319FD00021118BC
:101A00000E0615090904FF03FF0A03010155AA0187
:101A1000FFFFFFFFFF03FFFFFF25D0285004FF0259
:091A2000007AFF0101000300FF40
:101A4000234F76736B794D5232304150726F2320A1
:101A500023424C48454C492346333930232020202B
:101A60002020202020202020202020202020202076
:101C0000C2AFC2D353D9BF7581C043B20343FF8073
:101C1000752438752503B1C975EF0275E24043F1AB
:101C20008053A47F75D4FFD2877DFA780379E67C50
:101C300010752200752300901DD67B0675249875BB
:101C400025013087028142208708D8FBD9F9DCF7CB
:101C500081B4308708D8FBD9F9DCF781B4B189E4C5
:101C600093A3C39A6004DDC381B4DBDBB17B600264
:101C7000812B7B08E493FAA3B15CDBF87A30B15C8A
:101C8000752200752300B17BEAFCEBFDC3ED94FEE9
:101C9000400EB17B8A278B28ED30E0048A828B834B
:101CA000B17B7AC270D8C3ED94FE601350CEBD00F4
:101CB00025EC60097520007521FF0200008100A855
:101CC00027A9280809D804D90281D3B17FEA89AAB3
:101CD000F281C50D81A0C3ED94035049EDA2E092BD
:101CE000007AC5C3E5829400E583941C50902000DF
:101CF00010438F02438F0175B7A575B7F1F030001F
:101D00001FA827A9280809438F01538FFDD804D99C
:101D100002A12089AAE275B7A575B7F1F0A3A10DBC
:101D2000538FFC817C7AC1BD030CE493A3FAB140CC
:101D3000DCF8B138817C817EAA22AB23B15CEBFA5E
:101D4000EA6222752608C3E52313F523E52213F57D
:101D50002250066323A0632201D526EAB1C9B1C986
:101D600075260AEAF4200102D287300102C287B147
:101D7000C9C3134002C201D526EB22B17FEAFB2082
:101D80008702A17F308702A184752608AE24AF2583
:101D9000C3EF13FFEE13FEB1CDB1C9C3EA13308711
:101DA000024480FA30E703632201C3E52313F523DD
:101DB000E52213F52250066323A0632201D526D91C
:101DC000E52265236523F52222AE24AF250E0FDE22
:101DD000FEDFFCD20122424C48656C693437316326
:041DE000F390060175
:00000001FF
